:100000000C940E030C9452030C9452030C94520360
:100010000C9452030C9452030C9452030C9452030C
:100020000C9452030C9452030C94740E0C94460FCF
:100030000C9452030C9452030C9452030C945203EC
:100040000C9452030C9416220C9452030C945203F9
:100050000C9452030C94141D0C9452030C945203F0
:100060000C9452030C9452030C9452030C945203BC
:100070000C9452030C9452030C9452030C945203AC
:100080000C9452030C9452030C9452030C9452039C
:100090000C9452030C9452030C9452030C9452038C
:1000A0000C9452030C9452030C945203AB0FCD0FDB
:1000B000B810CD0FB8100F103210B81087109A106A
:1000C00074137413A313A313DB13FD132515251544
:1000D00008142515AF14AF1418152515251520156E
:1000E000BC14BC14BC14BC14BC14BC14BC14BC1490
:1000F000BC14BC14BC14BC14BC14BC14BC14BC1480
:10010000CE14DC14E314EA14F4146572676F646FA0
:10011000785F657A2F64656661756C74204020761F
:10012000342E302D3232322D67623835643266001B
:100130000000F0A12E004C002A00E1003541000033
:100140001E00140004001D6134004D001F001A0041
:1001500016001B00E1042A0020000800070006002A
:1001600050002C0021001500090019004F004A0022
:10017000220017000A0005000000656450000153CA
:100180000000006F0000E3004F0001530000006713
:100190000000E20023001C000B0011000000296198
:1001A000240018000D00100052004B0025000C0028
:1001B0000E00360051002800260012000F00370004
:1001C0002F002B00270013003342386130004E000F
:1001D0002D0031003468E500C1000000003001004E
:1001E00001000100010000003A001E02200222026C
:1001F000010001003B001F02210223020100010057
:100200003C002F0226022F00010001003D003002B9
:1002100027023000010001003E00310235003502A6
:1002200000000100010001000000010000000100C9
:100230000100010000000100000001003F00520029
:1002400051002402000001004000240021001E0093
:10025000010001004100250022001F0037000100BD
:100260004200260023002000270001004300250251
:100270002E0231002E000100440045000100010063
:100280000100000001000100010001000100000068
:100290000100010001000100010001000100010056
:1002A000F2000100010001000100F000F100010076
:1002B000F400010001000100F3000100F50001005D
:1002C0000100010001000100000001000100010027
:1002D0000000010000000100010001000000010019
:1002E0000000010001000100010001000000010008
:1002F0000100010001000100A9000100010001004E
:100300000100AC00AA00B600010001000100AB0032
:10031000A80001000100010001000100010001002E
:1003200001000100AE00010001000000000000001B
:10033000000000002A2B2800000000000000000040
:100340000000000000000029000000002C1E3420E6
:10035000212224342627252E362D3738271E1F200C
:100360002122232425263333362E37381F04050651
:100370000708090A0B0C0D0E0F1011121314151695
:100380001718191A1B1C1D2F3130232D3504050693
:100390000708090A0B0C0D0E0F1011121314151675
:1003A0001718191A1B1C1D2F3130354C0000000086
:1003B000000000000000000000000000000000003D
:1003C000000000000000000000000000000101012A
:1003D0000101010001010101000000000000000016
:1003E0000000000000000100010001010101010105
:1003F00001010101010101010101010101010101ED
:1004000001010101010101000000010100000000E3
:1004100000000000000000000000000000000000DC
:10042000000000000000000101010100160345006A
:10043000720067006F0044006F00780020004500E4
:100440005A00000016034500720067006F00440068
:100450006F007800200045005A00000004030904E2
:1004600009026D00040100A0FA0904000001030163
:100470000100092111010001224000070581030844
:10048000000A090401000103010200092111010011
:1004900001224D000705820308000A090402000139
:1004A0000300000009211101000122360007058325
:1004B0000308000A090403000103000000092111D8
:1004C0000100012239000705840310000112011008
:1004D0000100000008EDFE07130100010200010504
:1004E000010906A101050719E029E7150025019575
:1004F0000875018102050819012905950575019105
:10050000029501750391010507190029771500254A
:1005100001957875018102C005010980A10185025C
:1005200016010026B7001A01002AB70075109501C0
:100530008100C0050C0901A1018503160100269C5C
:10054000021A01002A9C02751095018100C0050164
:100550000902A1010901A1000509190129051500D8
:10056000250195057501810295017503810105013C
:10057000093009311581257F9502750881060938F2
:100580001581257F950175088106050C0A3802152D
:1005900081257F950175088106C0C005010906A166
:1005A00001050719E029E715002501950875018166
:1005B0000295017508810105081901290595057540
:1005C0000191029501750391010507190029FF1595
:1005D0000026FF00950675088100C000000000009D
:1005E000000000000000010204060A0F17202C3A48
:1005F0004A5D71879DB3C7DAE9F5FCFFFCF5E9DADE
:10060000C7B39D87715D4A3A2C20170F0A06040272
:1006100001000000000000000000000011241FBEC7
:10062000CFEFDAE0DEBFCDBF04B603FE24C0809179
:10063000FD019091FE01A091FF01B0910002873071
:10064000904BA740B04BB9F41092FD011092FE01FF
:100650001092FF011092000214BE84B7877F84BFFE
:1006600088E10FB6F89480936000109260000FBE8E
:10067000E0E0FFE3099511E0A0E0B1E0EAEBF7E488
:1006800002C005900D92A433B107D9F711E0A4E39D
:10069000B1E001C01D92AD3FB107E1F70E94BE0B72
:1006A0000C94DB230C9400001092B9008AE0809334
:1006B000B800089594EA9093BC009091BC0097FF15
:1006C000FCCF9091B900987F983021F0903111F0D3
:1006D00081E008958093BB0084E88093BC00809102
:1006E000BC0087FFFCCF8091B900887F883111F072
:1006F000803471F780E0089584E98093BC00809194
:10070000BC0084FDFCCF08958093BB0084E88093F7
:10071000BC008091BC0087FFFCCF9091B900987F0E
:1007200081E0983209F480E0089584E88093BC0069
:100730008091BC0087FFFCCF8091BB00089580B3FF
:100740008C7080BB81B3836F81BB08958091010160
:10075000811115C080E40E945A0380930101811128
:100760000CC082E10E94840380930101811105C0C5
:100770008FEF0E948403809301010E947C0384B167
:10078000807F84B985B1807F85B98AB1837F8AB93A
:100790008BB1837F8BB93E98469808950E946D0572
:1007A000809301010E94A6030E949F03E3E4F1E00D
:1007B000A5E3B1E011921D9281E0E135F807D1F790
:1007C0000C9457050E946D05809301010E94A603B9
:1007D0000E949F03E3E4F1E0A5E3B1E011921D92D2
:1007E00081E0E135F807D1F70895BF92CF92DF920B
:1007F000EF92FF920F931F93CF93DF9380910101AC
:10080000882379F0809134018F5F809334018111C6
:1008100008C00E946D0580930101811102C00E94F1
:10082000FF0405E311E0C0E0D0E0DD24D39482E0D2
:10083000C82EEE24E394F12CC73000F5809101011D
:10084000811162C080E40E945A03809301018111EA
:1008500012C082E10E9484038093010181110BC0C8
:10086000C7010C2E01C0880F0A94EAF780950E94F8
:100870008403809301010E947C0346C0CA30A1F02A
:1008800028F4C83059F0C93061F005C0CC3089F087
:1008900070F0CD3089F0209A289810C0219A2998BC
:1008A0000DC0229A2A980AC0239A2B9807C0529A00
:1008B00001C0539A5B9802C03E9A4698E0EAEA95D6
:1008C000F1F78FB179995AC092E081708D25892B0B
:1008D0007C9B02C090E001C094E0892B7D9B02C00C
:1008E00090E001C098E0892B7E9B02C090E001C09F
:1008F00090E1892B9FB19095991F9927991F929507
:10090000990F907E892B0FC08091010181114BC0FE
:1009100080E40E945A0380930101882389F1B12C5D
:100920000E947C038B2DF8019081981719F0808329
:10093000C09200010E94A60321960F5F1F4FCE3088
:10094000D10509F079CF80910001882371F18150A0
:1009500080930001882339F08FE99FE00197F1F738
:1009600000C0000022C0A3E4B1E0E5E3F1E0819122
:100970008D9391E0E334F907D1F717C090E0A5CF4C
:1009800083E10E948403809301018111C8CF81E437
:100990000E945A03809301018111C1CF0E949503E7
:1009A000B82EB094BDCF80E0BECF0E94FD0481E0A0
:1009B000DF91CF911F910F91FF90EF90DF90CF903B
:1009C000BF900895E82FF0E0ED5BFE4F8081089521
:1009D00008951F93CF93DF93C3E4D1E010E0899192
:1009E00090E00E94391C180F81E0C135D807B9F793
:1009F000812FDF91CF911F9108950C94CA055698CD
:100A00005E9825982D9826982E9827982F988FEFE6
:100A100090E0909389008093880090938B0080935E
:100A20008A0090938D0080938C00259A2D9A2FEF49
:100A300080E792E0215080409040E1F700C0000044
:100A4000269A2E9A2FEF80E792E021508040904026
:100A5000E1F700C00000279A2F9A2FEF80E792E07D
:100A6000215080409040E1F700C0000025982D986B
:100A70002FEF80E792E0215080409040E1F700C0E6
:100A8000000026982E982FEF80E792E021508040BA
:100A90009040E1F700C0000027982F9856985E9884
:100AA00025982D9826982E9827982F98089589EAAA
:100AB0008093800089E08093810024982C983F984F
:100AC0008AB18F748AB96E98479A8BB1806B8BB953
:100AD000769A0E94FF040C94C90580E2809301017C
:100AE0008091510181110EC00E94540381E08093D6
:100AF00051012FEF83ED90E3215080409040E1F7CA
:100B000000C0000080E40E945A038093010181111B
:100B10002EC00E94840380930101811128C00E948D
:100B2000840380930101811122C08FE30E9484031A
:100B30008093010181111BC00E947C0380E40E940C
:100B40005A0380930101811112C08CE00E9484033A
:100B50008093010181110BC00E94840380930101E5
:100B6000811105C08FE30E948403809301010E94DC
:100B70007C03809101010895611108C0FC0182810C
:100B8000882321F08AE091E00E94C30780E090E092
:100B9000089508956091BE017091BF018091C001D8
:100BA0009091C1010E94451C56985E9825982D98F9
:100BB00026982E9827982F98813019F0823021F0AE
:100BC0000895259A2D9A0895269A2E9A089581E0DF
:100BD000089581E008950C94E9050895282F88234D
:100BE00039F090E02A3010F44D9608950697089554
:100BF00087E290E00895BF92CF92DF92EF92FF924A
:100C00000F931F93CF93DF938C01FC01C081D1819F
:100C1000CE010E94C01ABE010E946D09EC01B8010C
:100C20000E94EB05882309F4A3C1F801828188237F
:100C3000C9F180915E0181111EC0C431F0E7DF0768
:100C400089F50E94ED0581E080935E010E94DF1C22
:100C500090935D0180935C011092550110925701B1
:100C600010925601109259011092580110925B0196
:100C700010925A017DC180915C0190915D010E94AA
:100C8000EB1C883C910570F480915501E82FF0E051
:100C9000EE0FFF1FEA5AFE4FD183C0838F5F809310
:100CA000550166C1C13020E8D20708F451C0F801EF
:100CB0008281882309F44CC06E01E894D7F88091B2
:100CC0005401813079F050F08230C1F482EE0E94FC
:100CD000121287E50E94121287E50EC082EE0E9472
:100CE00012120CC080EE0E94121281EE0E941212AB
:100CF00088E10E94121288E10E94DA128CE0E82E4C
:100D0000F12CC6010E2C02C0969587950A94E2F745
:100D10008F700E94EE05B82E0E9412128B2D0E9439
:100D2000DA12F4E0EF1AF1082CEFE2162FEFF206D8
:100D300041F780915401813029F010F0823041F464
:100D400082EE04C080EE0E94DA1281EE0E94DA1276
:100D5000C43180E7D80760F4C23090E7D90780F546
:100D6000C115E0E7DE0771F0C130D047F1F0EFC008
:100D7000C33320E7D20709F4BEC0C433D04709F417
:100D8000CEC0E5C0F8018281882309F4E5C00E9445
:100D90009315FFEF24E38CE0F15020408040E1F711
:100DA00000C000000E94391DE3C0F8018281882341
:100DB00009F4D2C08091DB0181608093DB01D8C04F
:100DC000F8018281882309F4C7C00E94941D811113
:100DD00002C00E947A1D0E94A71D90E09093EF012F
:100DE0008093EE01C230F0E7DF0721F48091EE013D
:100DF00081607AC0C33020E7D20721F48091EE01F0
:100E0000826072C0C43080E7D80721F48091EE017F
:100E100084606AC0C53090E7D90719F48091EE016B
:100E200027C0C630E0E7DE0721F48091EE01806143
:100E30005BC0C730F0E7DF0721F48091EE018062EC
:100E400053C0C83020E7D20721F48091EE018064BE
:100E50004BC0C93080E7D80721F48091EE0180684B
:100E600043C0CA3090E7D90729F48091EE0184602D
:100E700088603AC0CB30E0E7DE0721F48091EE01D4
:100E80008E7F32C0CC30F0E7DF0721F48091EE0195
:100E90008D7F2AC0CD3020E7D20721F48091EE016A
:100EA0008B7F22C0CE3080E7D80719F48091EE0105
:100EB0001AC08091EE01CF3090E7D90711F48F7EF0
:100EC00013C0C031E0E7DE0711F48F7D0DC0C131E2
:100ED000F0E7DF0711F48F7B07C0C231D04711F470
:100EE0008F7702C08B7F877F8093EE018091EE0128
:100EF0000E94AB1D3DC0F8018281882321F0109231
:100F0000520182E013C080915201811106C086E235
:100F10000E94121286E20E94DA1282E015C0F801E5
:100F20008281882331F01092530182E10E942913BB
:100F30001FC080915301811106C087E20E941212E6
:100F400087E20E94DA1282E10E94301311C081E030
:100F50008093520180935301C801DF91CF911F917B
:100F60000F91FF90EF90DF90CF90BF900C94E7052A
:100F700080E0DF91CF911F910F91FF90EF90DF9074
:100F8000CF90BF9008951F93CF93DF93EC01FE01A4
:100F900024912223F1F030E0F901E45DFC4F14913B
:100FA000F901E455FC4F2491222359F081EE0E946F
:100FB0001212812F0E941212812F0E94DA1281EEEA
:100FC00004C0812F0E941212812F0E94DA122196F2
:100FD000DECFDF91CF911F91089526E0729FF0013F
:100FE000112444E5849FE00DF11D1124E60FF11D4D
:100FF000EE0FFF1FEC5CFE4F859194910E947F09DC
:10100000811520E49207B0F5811540E3940708F0BC
:10101000DDC0803E9105D8F4803C910508F06BC09E
:10102000883A910578F4853A910508F06AC08130D4
:10103000910509F450C108F40DC18430910508F000
:101040004AC108C18B3B910508F466C003C18F3FBC
:10105000910509F048F4803F910508F0ACC0883E46
:10106000910508F438C1F6C0811520E2920708F016
:10107000A4C00895811543E5940790F4811522E5F5
:10108000920708F0C7C0811541E5940708F0BDC07C
:10109000811520E5920708F09CC09F70906A089522
:1010A000811545E59407D0F4811524E5920708F0F1
:1010B000C6C0282F2695269540E2249F9001112432
:1010C000AC014370552781E090E002C0880F991F62
:1010D0004A95E2F7822B932B9A680895811546E58D
:1010E000940708F4B1C09C0130562115304108F036
:1010F000B1C09F70ADC0FC01EE0FFF1FE055F04086
:1011000062C0853A910509F4A8C0863A910509F4B0
:10111000A7C083E890E40895883A910509F4A3C034
:10112000893A910509F4A2C08A3A910509F4A1C04F
:101130008B3A910509F4A0C08C3A910509F49FC03F
:101140008D3A910509F49EC0803B910509F49DC03C
:101150008E3A910509F49CC08F3A910509F49BC021
:10116000813B910509F49AC0823B910509F499C02D
:10117000833B910509F498C0843B910509F497C01D
:10118000853B910509F496C0863B910509F495C00D
:10119000873B910509F494C0883B910509F493C0FD
:1011A000893B910509F492C08A3B910509F091C0F1
:1011B0008AE296E40895906508959F70880F991FBC
:1011C000805D9E4FFC018591949108959927906CC4
:1011D0000895482F437021E030E002C0220F331FF2
:1011E0004A95E2F73C68AC0164E0569547956A95EC
:1011F000E1F74370342B8F708695869540E2849F8B
:10120000C0011124822B932B0895982F8827816F7A
:10121000906A0895282F2695269540E2249F9001F4
:101220001124AC014370552781E090E002C0880F83
:10123000991F4A95E2F7822B932B9C680895982F6B
:101240008827846F906A08958F719927982F88272F
:101250009062089580E090E0089581E890E4089518
:1012600082E890E4089582EE94E4089589EE94E48F
:1012700008958AEE94E4089585EB94E4089586EB4E
:1012800094E4089587EB94E408958CEC94E4089535
:101290008DEC94E4089583E895E408958AE895E454
:1012A000089582E995E4089584E995E4089581E23A
:1012B00096E4089583E296E4089584E296E408951E
:1012C00085E296E4089586E296E4089587E296E43E
:1012D000089580E094E40895089596E0799FF001E0
:1012E000112494E5899FE00DF11D1124E60FF11DF5
:1012F000EE0FFF1FEC5CFE4F8591949108958238AC
:10130000910549F1B0F48133910509F459C048F4CD
:101310008932910509F44FC08A32910509F455C00C
:1013200008958533910509F441C08933910599F0F9
:101330000895833E910531F138F4803E910591F096
:10134000823E9105A9F00895863E910501F1873E00
:10135000910539F108952091EE0120FD3BC021FD5A
:1013600039C008958091EE0180FF34C089E341C007
:101370008091EE0182FF32C08091EE0184FF2CC08B
:1013800080E037C08091EE0182FD28C0F5CF8091CA
:10139000EE0183FF25C08091EE0184FDF1CF87EE41
:1013A00028C08091EE0183FD1BC0F5CF8091EE0136
:1013B00085FF18C019C08091EE0185FF15C012C0CD
:1013C0008091EE0186FF12C013C08091EE0186FF6E
:1013D0000FC00CC080EE0DC083EE0BC082EE09C0C2
:1013E00086EE07C085E305C089E203C081E301C042
:1013F0008AE290E0089508950C94FB0980916F01B2
:101400000895CF93DF9300D01F92CDB7DEB7209120
:10141000F401243019F523E029839B838A832093E8
:10142000E9008FEF9091E800815095FD06C095EDA1
:101430009A95F1F700008111F5CF8091E80085FFC2
:101440000DC040E050E063E070E0CE0101960E94E4
:10145000670C8091E8008E778093E8000F900F90E2
:101460000F90DF91CF910895CF93DF9300D01F921B
:10147000CDB7DEB72091F401243021F522E0298395
:101480009B838A8383E08093E9008FEF9091E8004B
:10149000815095FD06C095ED9A95F1F700008111F8
:1014A000F5CF8091E80085FF0DC040E050E063E09B
:1014B00070E0CE0101960E94670C8091E8008E7763
:1014C0008093E8000F900F900F90DF91CF910895D7
:1014D0002091F4012430F1F422E02093E9002FEF71
:1014E0003091E800215035FD06C035ED3A95F1F711
:1014F00000002111F5CF2091E80025FF0BC040E04E
:1015000050E065E070E00E94670C8091E8008E7703
:101510008093E8000895CF93DF93EC018091F4016C
:10152000843009F046C090910C019923D9F0909134
:101530000D019923B9F08093E9008FEF9091E800B5
:10154000815095FD06C095E19A95F1F70000811153
:10155000F5CF8091E80085FF2CC040E050E060E1CD
:1015600070E017C081E08093E9008FEF9091E80070
:10157000815095FD06C095ED9A95F1F70000811117
:10158000F5CF8091E80085FF14C040E050E068E0AE
:1015900070E0CE010E94670C8091E8008E77809306
:1015A000E80080E1FE01AFE5B1E001900D928A957F
:1015B000E1F7DF91CF9108958091F301811109C086
:1015C0000E94F90D0E94560E8091E2008460809383
:1015D000E20008951092F301089508950C940322F7
:1015E0000E94D01C0E9409220E94F3100C94FC0956
:1015F00042E061EC81E00E94730D42E061EC82E028
:101600000E94730D42E061EC83E00E94730D42E1A1
:1016100061EC84E00C94730D8091F601833009F441
:1016200055C030F4813071F0823009F48EC00895D5
:101630008A3009F47AC08B3009F460C0893009F02F
:101640009CC020C08091F501813A09F096C080913C
:10165000E800877F8093E8008091F9019091FA017A
:10166000892B21F060E080E090E003C060E18FE52D
:1016700091E070E00E94B00C8091E8008B7780933D
:10168000E80008958091F501813209F076C08091DB
:10169000F9019091FA01009719F0039709F06DC0D4
:1016A0008091E800877F8093E8008091E80082FDC8
:1016B00005C08091F4018111F8CF5FC08091F100E5
:1016C00080936F018091E8008B7753C08091F50182
:1016D000813A09F052C08091F9019091FA01892B69
:1016E00009F04BC08091E800877F8093E8008091EB
:1016F000E80080FFFCCF80910C0136C08091F5019D
:101700008132D9F58091F9019091FA01892BA9F5DF
:101710008091E800877F8093E8000E94A80D809167
:10172000F70180930C010C9493158091F50181329F
:1017300021F58091E800877F8093E8000E94A80D42
:101740008091F8018093700108958091F501813AAC
:10175000A1F48091E800877F8093E8008091E80001
:1017600080FFFCCF809170018093F1008091E800B0
:101770008E778093E8000C94A80D089584B7877F36
:1017800084BF88E10FB6F8948093600010926000E7
:101790000FBE80E880936100109261000E944211A8
:1017A0000E94F90D0E94560E8091E20084608093A1
:1017B000E20078940E94D1100E94441182E091E0EE
:1017C0000E94EE100E94F1218091F401853069F4AD
:1017D0000E94981C8091F2018823B1F30E94C21CE0
:1017E000882391F30E94510CEFCF0E944A11ECCF55
:1017F000292F332723303105A9F06CF4213031052E
:1018000009F442C02230310509F043C08DE690E072
:1018100020E634E042C021323105C9F022323105E0
:1018200019F137C099278130910541F08230910537
:1018300041F0892B71F5ECE5F4E005C0E4E4F4E057
:1018400002C0ECE2F4E0849190E09F0126C0643095
:1018500000F5E62FF0E0EE0FFF1FEE5DFE4F20815A
:10186000318189E090E019C0643098F4E62FF0E00F
:10187000DF01AA0FBB1FA65EBE4F2D913C91EA5E11
:10188000FE4F808190E009C082E190E02DEC34E0D1
:1018900004C080E090E020E030E0FA013183208352
:1018A000089580E189BD82E189BD09B400FEFDCFC4
:1018B0008091D8008F7D8093D8008091E000826075
:1018C0008093E0008091E00081FDFCCF0895CF92ED
:1018D000DF92EF92FF920F931F93CF93DF937C01E0
:1018E0008B01EA010E94C90D811131C0209731F0AE
:1018F00088819981081B190BE80EF91EC12CD12C87
:101900000115110519F18091E80085FD14C0809141
:10191000E8008E778093E800209741F088819981D4
:101920008C0D9D1D9983888385E011C00E94C90D8F
:10193000882331F30CC0F70181917F018093F1007E
:1019400001501109FFEFCF1ADF0ADACF80E0DF91F3
:10195000CF911F910F91FF90EF90DF90CF9008955E
:101960002091FB013091FC012617370748F06115E3
:10197000710539F42091E8002E772093E80001C02A
:10198000B901FC0120E061157105B9F18091F40104
:10199000882309F440C0853009F43FC08091E800F5
:1019A00083FD3DC08091E80082FF06C08091E80081
:1019B00082FF26C080E008958091E80080FFE3CF99
:1019C0002091F3008091F20090E0922B6115710557
:1019D00051F08830910538F421912093F100615045
:1019E00071090196F3CF21E0089709F020E080917A
:1019F000E8008E778093E800C6CF2111C7CFD6CFFD
:101A00008091F401882339F0853039F08091E80025
:101A100083FFCCCF04C082E0089583E0089581E085
:101A200008952091FB013091FC012617370748F0FB
:101A30006115710539F42091E8002E772093E800B4
:101A400001C0B901FC0120E061157105C1F180916F
:101A5000F401882309F441C0853009F440C0809125
:101A6000E80083FD3EC08091E80082FF06C08091BF
:101A7000E80082FF27C080E008958091E80080FFA1
:101A8000E3CF2091F3008091F20090E0922B61155A
:101A9000710559F08830910540F424912093F100AC
:101AA0003196615071090196F2CF21E0089709F053
:101AB00020E08091E8008E778093E800C5CF211167
:101AC000C6CFD5CF8091F401882339F0853039F025
:101AD0008091E80083FFCBCF04C082E0089583E0CB
:101AE000089581E00895982F973058F59093E90074
:101AF000981739F07091EC002091ED005091F000B2
:101B000003C0242F762F50E021FF19C03091EB0045
:101B10003E7F3093EB003091ED003D7F3093ED0040
:101B20003091EB0031603093EB007093EC00209328
:101B3000ED005093F0002091EE0027FF07C09F5F5B
:101B4000D3CF8F708093E90081E0089580E00895FD
:101B50008091F50187FD05C08091E80080FF0EC0EF
:101B600012C08091E80082FD05C08091F4018111CE
:101B7000F8CF08958091E8008B7708C08091F40138
:101B80008111EACF08958091E8008E778093E80074
:101B900008958091E4009091E50045E62091EC00E5
:101BA00020FF21C02091E80020FD21C02091F401F8
:101BB000222389F0253089F02091EB0025FD0FC00C
:101BC0002091E4003091E5002817390739F341509E
:101BD00041F0C901E3CF82E0089583E0089581E0F8
:101BE000089584E008952091E80022FFDFCF80E08F
:101BF00008950E94670E0E946F0EE0EEF0E0808173
:101C000081608083E8EDF0E080818F77808319BC6C
:101C1000A7EDB0E08C918E7F8C9380818F7E808346
:101C20001092F30108950F931F93CF93DF930E94B7
:101C3000670E0E946F0EC8EDD0E088818F77888391
:101C400088818068888388818F7D888319BC109201
:101C5000F4011092F0011092F2011092F10100EEE5
:101C600010E0F80180818B7F808388818160888388
:101C700042E060E080E00E94730DE1EEF0E08081E0
:101C80008E7F8083E2EEF0E08081816080838081BE
:101C900088608083F80180818E7F80838881806165
:101CA0008883DF91CF911F910F910895E8EDF0E0C7
:101CB00080818F7E8083E7EDF0E08081816080838A
:101CC00084E082BF81E08093F3010C94130EE8ED71
:101CD000F0E080818E7F80831092E2000895109260
:101CE000DA001092E10008951F920F920FB60F9242
:101CF00011242F933F934F935F936F937F938F9311
:101D00009F93AF93BF93EF93FF938091E10082FF86
:101D10000BC08091E20082FF07C08091E1008B7FC1
:101D20008093E1000E94D0108091DA0080FF1FC0F4
:101D30008091D80080FF1BC08091DA008E7F809355
:101D4000DA008091D90080FF0DC080E189BD82E179
:101D500089BD09B400FEFDCF81E08093F4010E94AB
:101D6000DC0A05C019BC1092F4010E94EA0A8091B5
:101D7000E10080FF19C08091E20080FF15C08091D2
:101D8000E2008E7F8093E2008091E2008061809388
:101D9000E2008091D80080628093D80019BC85E071
:101DA0008093F4010E94EE0A8091E10084FF30C02C
:101DB0008091E20084FF2CC080E189BD82E189BD71
:101DC00009B400FEFDCF8091D8008F7D8093D800AC
:101DD0008091E1008F7E8093E1008091E2008F7E10
:101DE0008093E2008091E20081608093E200809124
:101DF000F001882311F084E007C08091E30087FFA1
:101E000002C083E001C081E08093F4010E94F00AE7
:101E10008091E10083FF29C08091E20083FF25C00B
:101E20008091E100877F8093E10082E08093F4015C
:101E30001092F0018091E1008E7F8093E10080910B
:101E4000E2008E7F8093E2008091E20080618093C7
:101E5000E20042E060E080E00E94730D8091F000BB
:101E600088608093F0000E94ED0AFF91EF91BF918E
:101E7000AF919F918F917F916F915F914F913F9122
:101E80002F910F900FBE0F901F9018951F920F92D9
:101E90000FB60F9211242F933F934F935F936F933D
:101EA0007F938F939F93AF93BF93CF93EF93FF93C2
:101EB000C091E900CF708091EC001092E900809110
:101EC000F000877F8093F00078940E94820F109238
:101ED000E9008091F00088608093F000C093E900F1
:101EE000FF91EF91CF91BF91AF919F918F917F9192
:101EF0006F915F914F913F912F910F900FBE0F9077
:101F00001F9018951F93CF93DF93CDB7DEB7AA9795
:101F10000FB6F894DEBF0FBECDBFE5EFF1E08091C4
:101F2000F100819321E0ED3FF207C9F70E940C0B0D
:101F30008091E80083FF1CC12091F5013091F601EA
:101F4000832F90E08A30910508F012C1FC01EA5A13
:101F5000FF4F0C948B23203881F0223809F008C100
:101F60008091F9018F708093E9008091EB0085FBEF
:101F7000882780F91092E90006C08091F1019091C4
:101F8000F201911182609091E800977F9093E800B0
:101F90008093F1001092F100C5C0822F8D7F09F06F
:101FA000E7C0222319F0223061F0E2C08091F701EE
:101FB000813009F0DDC0333009F080E08093F20118
:101FC00028C08091F701811124C02091F9012F7060
:101FD00009F4CEC02093E9008091EB0080FF19C086
:101FE0008091EB00333011F4806211C080618093E6
:101FF000EB0081E090E0022E01C0880F0A94EAF71E
:102000008093EA001092EA008091EB008860809350
:10201000EB001092E9008091E800877F86C02111D3
:10202000A7C01091F7011F778091E3008078812B82
:102030008093E3008091E800877F8093E8000E940E
:10204000A80D8091E80080FFFCCF8091E3008068BC
:102050008093E300112311F083E001C082E08093BC
:10206000F40186C02058223008F082C08091F70128
:102070009091F8018C3D23E0920779F583E08A8303
:102080008AE289834FB7F894DE01139620E03EE0A0
:1020900051E2E32FF0E050935700E49120FF03C09A
:1020A000E295EF703F5FEF708E2F90E0EA3010F016
:1020B000C79601C0C0968D939D932F5F243149F739
:1020C0004FBF8091E800877F8093E8006AE270E06C
:1020D000CE0101960E94B00C14C0AE014F5F5F4F5D
:1020E0006091F9010E94F80B009709F441C020911A
:1020F000E800277F2093E800BC0189819A810E9433
:10210000110D8091E8008B778093E80031C0203872
:1021100079F58091E800877F8093E8008091F00155
:102120008093F1008091E8008E778093E8000E9410
:10213000A80D1EC021111CC09091F7019230C0F46F
:102140008091E800877F8093E8009093F0010E94DF
:10215000A80D8091F001811104C08091E30087FFF8
:1021600002C084E001C081E08093F4010E94F80A7B
:102170008091E80083FF0AC08091E800877F809308
:10218000E8008091EB0080628093EB00AA960FB686
:10219000F894DEBF0FBECDBFDF91CF911F910895A0
:1021A0000895CF938091F4018823B1F08091E900E4
:1021B0008F709091EC0090FF02C090E801C090E019
:1021C000C92FC82B1092E9008091E80083FD0E947E
:1021D000820FCF70C093E900CF910895909376015C
:1021E000809375010895E0917501F0917601309723
:1021F00021F00190F081E02D099480E00895E091B4
:102200007501F0917601309721F00280F381E02D85
:1022100009940895E0917501F0917601309721F0CD
:102220000480F581E02D0994089520917301309187
:1022300074018217930771F0909374018093730176
:10224000E0917501F0917601309721F00680F781D9
:10225000E02D099408952091710130917201821747
:10226000930771F09093720180937101E091750171
:10227000F0917601309721F00084F185E02D0994EA
:10228000089508950C9441110E94D61C0E94CE031B
:102290000C945C1D9F92AF92BF92CF92DF92EF920F
:1022A000FF920F931F93CF93DF9300D000D000D005
:1022B000CDB7DEB70E94F50386E8E82E81E0F82E60
:1022C0000DE010E0CC24C394D12C902E802F0E94DE
:1022D000E204F701B2907F01B826A1F40150110980
:1022E000A0F78FEF89838A831B820E94DF1C8160A5
:1022F000782F9D838C8349815A816B818D810E94C7
:10230000E41131C09091DB0191FF04C08E830E94E3
:10231000E8048E8125E030E0A601022E01C0440FC2
:102320000A94EAF7A42E4B21D1F029839A828A21BC
:1023300091E009F490E09B830E94DF1C8160782F7C
:102340009D838C8349815A816B818D810E94E41128
:10235000F801E858FE4F80818A25808304C021500F
:102360003109D0F6BBCF0E94291F109177010E943E
:10237000F3101817B9F00E94F31080937701269696
:102380000FB6F894DEBF0FBECDBFDF91CF911F9186
:102390000F91FF90EF90DF90CF90BF90AF909F9004
:1023A0000C94FC0926960FB6F894DEBF0FBECDBF85
:1023B000DF91CF911F910F91FF90EF90DF90CF9021
:1023C000BF90AF909F900895CF93DF93CDB7DEB7C6
:1023D0002B970FB6F894DEBF0FBECDBF4F83588743
:1023E00069877A878B87DE01119686E0FD0111925D
:1023F0008A95E9F785E0FE01379601900D928A955E
:10240000E1F749815A816B817C818D819E810E9497
:1024100063182B960FB6F894DEBF0FBECDBFDF91C9
:10242000CF910895CF93C82F882309F4C1C0823873
:1024300059F40E94F31081FDBBC089E30E94401B48
:102440000E940A1C89E30CC0833879F40E94F310BF
:1024500080FDAEC083E50E94401B0E940A1C83E5FC
:102460000E94801BCF910C940A1C843859F40E945E
:10247000F31082FD9DC087E40E94401B0E940A1C4D
:1024800087E4EECF8CEF8C0F813A48F48C2F0E94BA
:10249000592181118DC08C2F0E94401BE3CF80E217
:1024A0008C0F883048F4C77081E001C0880FCA954E
:1024B000EAF70E94C11BD6CF8BE58C0F833078F4EE
:1024C000C53A29F0C63A31F482E890E005C081E8C7
:1024D00090E002C083E890E0CF910C94151188E55C
:1024E0008C0F833108F064C0C83A39F1C93A41F120
:1024F000CA3A49F1CB3A51F1CC3A59F1CD3A61F1AE
:10250000C03B69F1CE3A71F1CF3A79F1C13B81F12B
:10251000C23B89F1C33B91F1C43B99F1C53BA1F1A9
:10252000C63BA9F1C73BB1F1C83BB9F1C93BC1F109
:10253000CA3BC9F58AE292E038C082EE90E035C02D
:1025400089EE90E032C08AEE90E02FC085EB90E0FB
:102550002CC086EB90E029C087EB90E026C08CEC85
:1025600090E023C08DEC90E020C083E891E01DC096
:102570008AE891E01AC082E991E017C084E991E00D
:1025800014C081E292E011C083E292E00EC084E2C6
:1025900092E00BC085E292E008C086E292E005C0BE
:1025A00087E292E002C080E090E0CF910C942B1182
:1025B000CF910895882309F44BC0823859F40E94C2
:1025C000F31081FF45C089E30E94401B0E940A1C52
:1025D00089E30CC0833871F40E94F31080FF38C087
:1025E00083E50E94401B0E940A1C83E50E94801B19
:1025F0000C940A1C843859F40E94F31082FF28C0FE
:1026000087E40E94401B0E940A1C87E4EFCF9CEFE6
:10261000980F913A58F390E2980F983050F48770E1
:1026200091E001C0990F8A95EAF7892F0E94C71B94
:10263000DFCF9BE5980F933020F480E090E00C947E
:102640001511885A833120F480E090E00C942B110E
:102650000895882321F00E94C11B0C940A1C089540
:10266000882321F00E94C71B0C940A1C08958F92A6
:102670009F92AF92BF92CF92DF92EF92FF920F9311
:102680001F93CF93DF931F92CDB7DEB74C01A62ED9
:10269000472FFC01E580E2948FE0E822F280FF20E2
:1026A00021F079830E94DE1B498149830E94391BF6
:1026B0004981882381F0FF2071F080E28A0D883003
:1026C00050F082E00E94221B0E94391BBB24B3946D
:1026D000B826498101C0B12CE42FE295EF70F0E0FB
:1026E000E05AFF4F0C948B23842F807F142F1F7090
:1026F000882311F01295107FFF2089F0112309F42F
:102700008DC180E28A0D883020F4812F0E94C11B88
:1027100003C0812F0E94D11B0E940A1C7FC18A2DF9
:102720000E94DA12112309F490C180E28A0D8830E8
:1027300020F4812F0E94C71B03C0812F0E94D71B4A
:102740000E940A1C82C1242F207F842F8F70203288
:1027500011F08295807FAA2021F0F1E0AF16B9F048
:1027600020C0FF2049F0EE2009F40FC191E0E912EA
:102770000CC10E94F11B69C1EE2021F0E1E0EE16D0
:1027800009F463C189830E94F41B898104C1FF207D
:1027900029F0F1E0FE1508F458C1F7C0E11055C169
:1027A000FAC0FF2021F0EE2009F4EFC037C1EE207F
:1027B00009F4F1C039C1242F26952695237030E005
:1027C0002115310521F02130310561F03EC1FF2096
:1027D00021F08A2D942F937002C080E090E00E9437
:1027E000151133C1FF2021F08A2D942F937002C060
:1027F00080E090E00E942B1128C18A2DFF2019F063
:102800000E94311E02C00E94991E0E941E1F1DC1FF
:10281000842F837009F04EC0F11017C12A2D229524
:1028200026952770220F220F8A2D8F70C82ED12C4B
:10283000E12CF12C022E04C0CC0CDD1CEE1CFF1C84
:102840000A94D2F7A4FE10C06FE070E080E090E040
:1028500004C0660F771F881F991F2A95D2F76095CD
:1028600070958095909503C060E070E0CB01242FB7
:1028700026952695237030E02230310569F023300B
:10288000310589F06C297D298E299F292130310558
:1028900071F00E94B719D9C06C297D298E299F2912
:1028A0000E94D119D2C00E94B719C701B6010E9477
:1028B0009D19CBC0FF2019F0842F817001C086952F
:1028C000882309F4C2C02A2D229526952770220F4D
:1028D000220F8A2D8F70C82ED12CE12CF12C022EC4
:1028E00004C0CC0CDD1CEE1CFF1C0A94D2F7A4FE25
:1028F00010C06FE070E080E090E004C0660F771FCA
:10290000881F991F2A95D2F76095709580959095AC
:1029100003C060E070E0CB01242F2695269523703C
:1029200030E02230310569F02330310589F06C291F
:102930007D298E299F292130310571F00E948B1A43
:1029400084C06C297D298E299F290E94A51A7DC0EB
:102950000E948B1AC701B6010E94711A76C00A2D17
:1029600010E0F801E05EF109E531F10508F052C030
:10297000E059FF4F0C948B231A2D1F70842F8F71F9
:10298000FF2031F00E940A1A812F0E9429135DC096
:102990000E942B1A812F0E94301357C0FF2039F05C
:1029A000E11053C0842F8F710E94501A4EC081E0F5
:1029B0008E1508F44AC0F6CFFF2039F0842F8F71AE
:1029C0000E940A1A42C0FF20C9F3842F8F710E940F
:1029D0002B1A3BC0FF2029F0842F8F710E94F5191C
:1029E00034C00E94EB1931C0FF2051F0142F1F7129
:1029F000812F0E940A1A63E0812F0E94191B25C0B3
:102A000081E00E94221B91E09E15F8F482E00E9472
:102A1000221B1BC0FF2031F0EE2081F28A2D0E9484
:102A2000121213C0EE2089F28A2D0E94DA120DC014
:102A30004F706A2DC4010E94BC050E94101905C088
:102A40004F706A2DC4010E946C09BB20F1F00E94F6
:102A5000151B80FD1AC0F40112820E940F1B0E94F8
:102A60000A1AC4010E9453150E940F1B0F90DF9198
:102A7000CF911F910F91FF90EF90DF90CF90BF907B
:102A8000AF909F908F900C942B1A0F90DF91CF9165
:102A90001F910F91FF90EF90DF90CF90BF90AF907C
:102AA0009F908F9008950F931F93CF93DF93EC0126
:102AB000288139818B819C81892B31F03F3F11F036
:102AC00080E003C02F3FE1F781E0811113C0CE0108
:102AD0000E94FB05882371F0688179818A810E94B8
:102AE0000B1B8C010E94BF1A0E949219B801CE01E3
:102AF0000E943713DF91CF911F910F9108950E948B
:102B0000DE1B0E94EE1B0E94B31B0E940A1C0E9447
:102B1000CA1F0E941E1F80E090E00E94151180E0F5
:102B200090E00C942B110E94CE1B0C947F150E94F8
:102B3000001B292F22952F7030E02C3031054CF4EA
:102B40002A3031056CF42250310922303105B0F4BD
:102B500007C02C30310571F02F30310559F00EC00F
:102B6000803F31F018F4803E48F402C0843F31F4D5
:102B700081E0089593FB882780F9089580E0089507
:102B8000CF93DF9300D000D01F92CDB7DEB70F9068
:102B90000F900F900F900F90DF91CF910895CF93EA
:102BA000DF9300D000D000D0CDB7DEB726960FB6A9
:102BB000F894DEBF0FBECDBFDF91CF9108951F9374
:102BC000CF93DF93C091860116E080918701C817EB
:102BD00099F0D0E01C9FF0011D9FF00D1124E857E3
:102BE000FE4F4081518162817381848195810E9471
:102BF000CF152196C770E9CFDF91CF911F9108952E
:102C00004091B8015091B9016091BA017091BB0136
:102C10008091BC019091BD010C94CF15CF93809110
:102C2000BD0182958F7009F05FC08091BA01882341
:102C300009F45AC020918601A09187016091B801E2
:102C40007091B9018091BB019091BC0131E06F3F5F
:102C500009F030E0B32FC6E02A1709F445C0009709
:102C600021F07F3F21F44B2F03C041E001C040E041
:102C700030E040FD35C0C29FF001C39FF00D11242C
:102C8000E857FE4F418174132BC04081641328C064
:102C90004281411125C0438154814817590710F4DE
:102CA00041505109481B590B483C5105C8F48091CB
:102CB000BD018F7080618093BD0186E0829FF0012D
:102CC000839FF00D1124E357FE4F80818F70806148
:102CD000808388EB91E00E945315CF910C94DF150F
:102CE0002F5F3F4F2770B8CFCF910895CF92DF92DB
:102CF000EF92FF920F931F93CF93DF93CDB7DEB781
:102D000062970FB6F894DEBF0FBECDBF8C0185E091
:102D1000F801DE011D9601900D928A95E1F7D80128
:102D20004C9111965C91119712966C911297139693
:102D3000ED90FC9014977091B801E091B901209149
:102D4000BB013091BC012115310531F0EF3F31F469
:102D500081E07F3F19F403C081E001C080E0B82F1B
:102D6000B170CB2E80FD6CC1D090BA01DD2009F48A
:102D7000F5C0F091BD01E216F30638F0C701821BE1
:102D8000930B883C910548F09BC0209530952E0D03
:102D90003F1D283C310508F093C08F2F807F09F03C
:102DA00052C0E51314C0741312C0D62E61110FC0A7
:102DB000FF70F061F093BD010E94001688EB91E076
:102DC0000E9453158091BD01F80185836CC1EF28E5
:102DD00031F05F3F31F481E04F3F19F403C081E0EF
:102DE00001C080E080FD03C081E0862701C080E053
:102DF000F82FF170FF2E80FF1CC08091860120917A
:102E0000870136E0821709F428C190E0389FF0016D
:102E1000399FF00D1124E857FE4F7181571306C0FA
:102E20007081471303C07281671303C001968770D6
:102E3000E9CFD62E662309F436C18091BD018160A9
:102E40008093BD0153C0E51308C0741306C061111F
:102E500004C0D8011596FC93AEC04D875E878D8562
:102E60009E856A8B0E9497156A89882329F1D62E40
:102E7000662311F12091BD01822F82958F7090E021
:102E800002970CF460C08091B8019091B9019887C5
:102E90008F831986FB86EA862C87CE01079651C060
:102EA000E51731F14D875E878D859E856A8B0E947F
:102EB00097156A8981112EC0C8010E945315A4C0BC
:102EC0008F2F807F69F77E2DF98AE88A89890E9491
:102ED000C01588EB91E00E945315E8EBF1E086E025
:102EE000DF011D928A95E9F70E940016D12CDBC004
:102EF0007413D8CF6111D6CFD8011596FC93C801B1
:102F00000E945315E8EBF1E086E0DF011D928A95FF
:102F1000E9F7C9C0D62E662379F22091BD01822F30
:102F200082958F7090E0029774F08091B801909133
:102F3000B9019A8389831B82FD82EC822E83CE01A4
:102F400001960E94531586E0F801A8EBB1E00190CC
:102F50000D928A95E1F70E940E166FC0E216F306F5
:102F600028F0C701821B930B9C0104C0209530956B
:102F70002E0D3F1D283C310508F052C0D62E662389
:102F800009F49ACFE5132CC074132AC08091BD01B7
:102F900080FD1DC0982F92959F70C9F0D80115969D
:102FA0008C9315979F3039F09F5F9295907F8F702B
:102FB000892B15968C93C8010E94531586E0F80161
:102FC000A8EBB1E001900D928A95E1F736C086E05A
:102FD000F801A8EBB1E001900D928A95E1F763C08A
:102FE0004D875E878D859E850E949715882379F091
:102FF00086E0F801A8EBB1E001900D928A95E1F727
:103000000E940E160E940016DD24D3944CC08091BD
:10301000BD0181608093BD01C8010E94531543C06A
:103020007E2DF98AE88A89890E94C015E8EBF1E0D3
:1030300086E0DF011D928A95E9F70E94001633C0F1
:10304000662309F439CF4D875E878D859E850E9462
:103050009715882309F430CFCBCF4D875E878D85B8
:103060009E850E94001B292F22952F7030E0223070
:1030700031052CF49F7041F0811106C00CC0243042
:1030800031052CF49F7049F4805E883020F0C8012F
:103090000E945315CF2CDC2C06C0D80115969C91AC
:1030A000907F91F7F8CF8D2D62960FB6F894DEBF22
:1030B0000FBECDBFDF91CF911F910F91FF90EF9089
:1030C000DF90CF9008951F93CF93DF93CDB7DEB7F6
:1030D0002C970FB6F894DEBF0FBECDBF4F83588735
:1030E00069877A878B879C87CE0107960E94761620
:1030F0008823C1F02F8138858A859B85892B31F003
:103100003F3F11F080E003C02F3FE1F781E08111E4
:1031100047C04F81588569857A858B859C850E943B
:10312000CF153EC086E0FE013796DE011196019074
:103130000D928A95E1F7FF81E8854A855B85411507
:10314000510531F0EF3F31F481E0FF3F19F403C046
:1031500081E001C080E080FD23C02091870130E044
:10316000C9010196877099276091860170E08617E2
:103170009707F1F1F983EA835D834C8396E0929F90
:10318000D001939FB00D1124A857BE4FFE01319678
:1031900001900D929A95E1F7809387010E94DF15C7
:1031A00016E08091860190918701891779F1189F27
:1031B000C001112488579E4F0E947616882331F152
:1031C000E09186011E9FF0011124E857FE4F4081D7
:1031D000518162817381848195810E94CF15809194
:1031E000860190E001968770992780938601D9CF58
:1031F0000E9493151092870110928601E8EBF1E08E
:1032000086E0DF011D928A95E9F7CACF2C960FB6AA
:10321000F894DEBF0FBECDBFDF91CF911F9108950F
:10322000EF92FF920F931F93CF93DF939C01009730
:1032300009F471C0F12CEE24E394E9012196F9011F
:103240008491843740F4843008F056C0813081F096
:10325000823021F160C0853709F449C0C0F19CE794
:10326000980F903708F057C08F770E94DA1246C047
:1032700089010E5F1F4FFE01849190E2980F9830F4
:1032800050F48770FE2D01C0FF0F8A95EAF78F2F4B
:103290000E94E11B15C00E94121214C089010E5F2A
:1032A0001F4FFE01849190E2980F983068F4877068
:1032B000FE2D01C0FF0F8A95EAF78F2F0E94E71BB2
:1032C0000E940A1CE8011AC00E94DA12FBCF2E5F8E
:1032D0003F4FFE01C491CC2341F08FE99FE001975D
:1032E000F1F700C00000C150F6CFE90107C0FE01B0
:1032F000F490E901229602C00E9412128F2D8823B9
:1033000041F0EFE9FFE03197F1F700C00000815094
:10331000F6CF9E0192CFDF91CF911F910F91FF9039
:10332000EF90089508956093C2017093C301809354
:10333000C4019093C5010C947F150F931F930091C6
:10334000C2011091C3012091C4013091C501062B27
:10335000172B282B392B0093C2011093C301209304
:10336000C4013093C5011F910F910C947F150F93E9
:103370001F930091C2011091C3012091C4013091AB
:10338000C50106231723282339230093C201109374
:10339000C3012093C4013093C5011F910F910C9478
:1033A0007F150F931F930091C2011091C3012091CB
:1033B000C4013091C5010627172728273927009314
:1033C000C2011093C3012093C4013093C5011F9122
:1033D0000F910C947F151092BE011092BF011092B4
:1033E000C0011092C1010C947F1541E050E060E0F3
:1033F00070E004C0440F551F661F771F8A95D2F7EF
:103400004093BE015093BF016093C0017093C1010E
:103410000C947F1541E050E060E070E004C0440F80
:10342000551F661F771F8A95D2F78091BE01909134
:10343000BF01A091C001B091C101842B952BA62B97
:10344000B72B8093BE019093BF01A093C001B093AE
:10345000C1010C947F1541E050E060E070E004C0D1
:10346000440F551F661F771F8A95D2F740955095D8
:10347000609570958091BE019091BF01A091C001AF
:10348000B091C10184239523A623B7238093BE0165
:103490009093BF01A093C001B093C1010C947F151C
:1034A00041E050E060E070E004C0440F551F661F2B
:1034B000771F8A95D2F78091BE019091BF01A091AC
:1034C000C001B091C10184279527A627B727809313
:1034D000BE019093BF01A093C001B093C1010C94B1
:1034E0007F150F931F930091BE011091BF01209192
:1034F000C0013091C101062B172B282B392B0093CB
:10350000BE011093BF012093C0013093C1011F91F0
:103510000F910C947F150F931F930091BE01109192
:10352000BF012091C0013091C10106231723282338
:1035300039230093BE011093BF012093C001309343
:10354000C1011F910F910C947F150F931F93009150
:10355000BE011091BF012091C0013091C101062729
:103560001727282739270093BE011093BF01209306
:10357000C0013093C1011F910F910C947F150895E4
:10358000CF92DF92EF92FF920F931F93CF93DF932F
:10359000EC01C090C201D090C301E090C401F09052
:1035A000C5018091BE019091BF01A091C001B09171
:1035B000C101C82AD92AEA2AFB2A0FE110E0B70183
:1035C000A601002E04C076956795579547950A94F5
:1035D000D2F740FD05C00150110988F780E007C00F
:1035E000BE01802F0E94ED070197A9F3802FDF9184
:1035F000CF911F910F91FF90EF90DF90CF900895A2
:10360000CF93DF93EC010E94C01ABE010E94ED0728
:10361000DF91CF910895CB010E94001B0895809106
:10362000C60185958595859508958091C601877019
:10363000089598E0899F90011124622B6093C60140
:103640000C940A1A4091C601809584238093C60188
:10365000982F977069F450E0282F332727FD309575
:103660004217530729F08595859585950C942B1A5B
:1036700008959091C601977081E009F480E0089563
:1036800090910C019923D9F090910D019923B9F0F3
:10369000982F9695969596959F3088F5E0910E0116
:1036A000F0910F01E90FF11D877021E030E001C0BA
:1036B000220F8A95EAF78181822B818308954091B8
:1036C0000E0150910F0120E030E09FEFFA01E20F70
:1036D000F31F6281681799F09F3F19F4611101C0CF
:1036E000922F2F5F3F4F2E30310581F79F3F39F0EA
:1036F000FA01E90FF11D97FDFA9582830895089567
:1037000090910C019923E1F090910D019923C1F062
:10371000982F9695969596959F3020F5E0910E01FD
:10372000F0910F01E90FF11D877021E030E001C039
:10373000220F8A95EAF72095818128232183089515
:1037400040910E0150910F0120E030E0FA01E20FAC
:10375000F31F9281981301C012822F5F3F4F2E30CA
:103760003105A1F7089581E090E0E0910E01F0911C
:103770000F01E80FF91F1082019680319105A9F71A
:1037800008959091DA01982B9093DA01089580952D
:103790009091DA0198239093DA0108951092DA015A
:1037A00008959091D901982B9093D901089580950F
:1037B0009091D90198239093D90108951092D9013D
:1037C00008959091D801982B9093D80108958095F1
:1037D0009091D80198239093D80108951092D80120
:1037E00008958093C70108951092C70108954091EC
:1037F0000E0150910F0120E030E080E0FA01E20F6D
:10380000F31F918191118F5F2F5F3F4F2F30310553
:10381000A9F70895E0910E01F0910F018091DA016E
:103820008083E0910E01F0910F0180819091D90188
:10383000892B8083E0910E01F0910F01808190919E
:10384000D801892B80839091C701992361F0E09181
:103850000E01F0910F018081892B80830E94F71B5C
:1038600081111092C70180910E0190910F010C946B
:10387000FF1040E0009739F09C012150310982236C
:1038800093234F5FF7CF842F0895CF92DF92EF926B
:10389000FF920F931F936C01EE24FF24C114D104F7
:1038A000E104F10421F46B017C0180E001C080E1BE
:1038B00033272F2D1E2D0D2D011511052105310545
:1038C00019F0885F6801790197018601A4E03695B7
:1038D000279517950795AA95D1F70115110521058B
:1038E000310519F08C5F6801790197018601F2E0DA
:1038F0003695279517950795FA95D1F70115110576
:103900002105310519F08E5F68017901B701A60123
:103910007695679557954795452B462B472B09F08C
:103920008F5F1F910F91FF90EF90DF90CF900895E0
:103930008091F401843021F11092DC0120E488E1CF
:1039400090E00FB6F894A895809360000FBE209386
:10395000600080E00E94FC0983B7817F846083BFA0
:1039600083B7816083BF7894889583B78E7F83BF48
:1039700088E10FB6F89480936000109260000FBE4B
:10398000089508950E94E2030E94F5030E94C11C5D
:103990000E94E90491E0811101C090E0892F08950F
:1039A0000E9493150E94F3100C94FC0982E084BDE0
:1039B00093E095BD9AEF97BD80936E0008952FB761
:1039C000F8948091DD019091DE01A091DF01B0912A
:1039D000E0012FBF0895CF92DF92EF92FF920F93F5
:1039E0001F932FB7F8944091DD015091DE01609153
:1039F000DF017091E0012FBF6A017B01EE24FF24FB
:103A00008C0120E030E0C016D106E206F30610F487
:103A100041505109481B590BCA011F910F91FF904A
:103A2000EF90DF90CF9008951F920F920FB60F92F4
:103A300011248F939F93AF93BF938091DD01909159
:103A4000DE01A091DF01B091E0010196A11DB11D41
:103A50008093DD019093DE01A093DF01B093E0013C
:103A6000BF91AF919F918F910F900FBE0F901F90BC
:103A700018950E94F90DF8942FEF87EA91E62150EE
:103A800080409040E1F700C0000087E090EBDC014F
:103A90008093FD019093FE01A093FF01B09300027B
:103AA0002CE088E190E00FB6F894A8958093600030
:103AB0000FBE20936000FFCF0E94941D811102C0B1
:103AC0000E947A1D0E949F1D8093DB010E94A71D0A
:103AD00090E09093EF018093EE0187FB882780F9B7
:103AE00080930D010E94A31D682F70E080E090E09C
:103AF0000C9493196DEE7EEF80E090E00E94C52358
:103B000060E082E090E00E94B32360E083E090E018
:103B10000E94B32360E084E090E00E94B32360E061
:103B200085E090E00C94B32380E090E00E94AD2308
:103B300021E08D3E9E4F09F020E0822F089582E023
:103B400090E00C94A52383E090E00C94A52384E0FE
:103B500090E00C94A523682F84E090E00C94B323AC
:103B60008091E30180FF0BC06091130185E0689FA5
:103B7000B001112475956795759567952AC081FFE9
:103B800009C06091130185E0689FB001112475950B
:103B900067951FC082FF07C06091130185E0689F91
:103BA000B001112416C04091E4014423C9F0609192
:103BB0001201461788F72091130185E0289F900194
:103BC0001124429FC001439F900D112470E00E9478
:103BD00077236038710540F46115710539F002C032
:103BE00065E070E0862F08958FE7089581E00895DD
:103BF0008091E30180FF08C06091110170E075952C
:103C000067957595679521C081FF06C06091110188
:103C100070E07595679519C082FF04C0609111012D
:103C200070E010C08091E4018823C1F06091100120
:103C30008617A0F790911101989FC001112470E0A0
:103C40000E9477236038710528F46115710521F011
:103C5000862F08958FE7089581E0089561E070E070
:103C6000F4CF803F21F40E94B01D819504C0813FB4
:103C700029F40E94B01D8093E7010895823F21F44A
:103C80000E94B01D819504C0833F29F40E94B01D9D
:103C90008093E6010895893F19F40E94F81D05C03C
:103CA0008A3F31F40E94F81D81958093E8010895C0
:103CB0008B3F21F40E94F81D819504C08C3F29F4AC
:103CC0000E94F81D8093E9010895843F21F48091BA
:103CD000E501816017C0853F21F48091E501826094
:103CE00011C0863F21F48091E50184600BC0873FBD
:103CF00021F48091E501886005C0883F31F480910E
:103D0000E50180618093E50108958D3F21F4809164
:103D1000E30181600BC08E3F21F48091E30182605A
:103D200005C08F3F29F48091E30184608093E30113
:103D30000895803F39F48091E70187FF6CC01092AD
:103D4000E70169C0813F29F48091E7011816BCF3AF
:103D500062C09091E601823F29F497FF5CC0109207
:103D6000E60159C0833F19F41916CCF354C0893FBA
:103D700041F48091E80118160CF04DC01092E80152
:103D80004AC08A3F29F48091E80187FF44C0F6CFFA
:103D90008B3F39F48091E90187FF3DC01092E90122
:103DA0003AC08C3F29F48091E9011816BCF333C066
:103DB000843F21F48091E5018E7F17C0853F21F477
:103DC0008091E5018D7F11C0863F21F48091E5014E
:103DD0008B7F0BC0873F21F48091E501877F05C071
:103DE000883F31F48091E5018F7E8093E50113C017
:103DF0008D3F21F48091E3018E7F0BC08E3F21F433
:103E00008091E3018D7F05C08F3F29F48091E3010C
:103E10008B7F8093E3018091E60181110EC0809138
:103E2000E70181110AC08091E801811106C08091EB
:103E3000E901811102C01092E401089585EE91E03C
:103E40000E940A110E94DF1C9093E2018093E1011D
:103E500008951F93CF93DF938091E1019091E20148
:103E60000E94EB1C4091E401442321F020911401B5
:103E700030E006C0209115015AE0259F90011124E1
:103E80008217930708F482C08091E6011091E70140
:103E9000D091E801C091E901811107C0111105C05D
:103EA000D11103C0CC2309F471C04F3F19F04F5F0B
:103EB0004093E401181624F40E94B01D8093E6019B
:103EC0008091E60187FF05C00E94B01D8195809317
:103ED000E601111624F40E94B01D8093E701809141
:103EE000E70187FF05C00E94B01D81958093E7011F
:103EF0006091E601662339F11091E701112319F170
:103F0000772767FD7095872F972F0E94882223E3DC
:103F100033E343E35FE30E94EC220E945522609367
:103F2000E601612F772767FD7095872F972F0E94F5
:103F3000882223E333E343E35FE30E94EC220E9401
:103F400055226093E7011D1624F40E94F81D80930A
:103F5000E8018091E80187FF05C00E94F81D819566
:103F60008093E8011C1624F40E94F81D8093E90157
:103F70008091E90187FF05C00E94F81D819580931B
:103F8000E901DF91CF911F910C941E1FDF91CF911A
:103F90001F910895E5EEF1E085E0DF011D928A951D
:103FA000E9F71092E4011092E3010895833081F162
:103FB00028F4813059F08230D1F00895853009F429
:103FC00049C0B8F1863009F456C008952091150112
:103FD000862F90E0820F911D8F3F910520F4620F94
:103FE0006093150108958FEF809315010895209136
:103FF0001401862F90E0820F911D8F3F910520F4D0
:10400000620F6093140108958FEF80931401089557
:1040100020911301862F90E0820F911D8F3F910513
:1040200020F4620F6093130108958FEF80931301C2
:10403000089520911201862F90E0820F911D8F3FED
:10404000910520F4620F6093120108958FEF809321
:104050001201089520911101862F90E0820F911D89
:104060008F3F910520F4620F6093110108958FEF47
:1040700080931101089520911001862F90E0820F06
:10408000911D8F3F910520F4620F609310010895F8
:104090008FEF809310010895833011F128F481305F
:1040A00049F0823091F00895853081F120F1863019
:1040B000C1F1089580911501681720F4861B809343
:1040C0001501089510921501089580911401681743
:1040D00020F4861B80931401089510921401089512
:1040E00080911301681720F4861B809313010895B3
:1040F00010921301089580911201681720F4861B15
:104100008093120108951092120108958091110177
:10411000681720F4861B80931101089510921101F5
:10412000089580911001681720F4861B8093100178
:1041300008951092100108958D3109F43FC008F5DB
:10414000803109F485C070F4873009F456C018F442
:104150008630D9F131C08B3009F4A5C08E3009F416
:1041600066C02AC0863109F49EC020F4813109F46A
:1041700079C022C0893109F496C08B3109F44DC051
:104180001BC0853309F487C048F4873209F483C023
:1041900008F473C0893209F47EC00EC0833438F449
:1041A0008A3308F068C0883309F47DC005C08334C1
:1041B00009F471C0883499F080E008950E940F22BC
:1041C0000E94F3100E94FC096EC08091DB01817F88
:1041D0008E7F8093DB0181E08093EB0108950E9444
:1041E00093152FEF83ED90E3215080409040E1F74D
:1041F00000C000000E94391D56C09091DB01892F3C
:104200008095817080FB90F919F0966098601DC0D0
:10421000997F977F9093DB0146C09091DB0191FBE2
:10422000882780F921E0822780FB91F909C09091CD
:10423000DB0192FB882780F921E0822780FB92F93D
:104240009093DB01882379F191609093DB010895CD
:104250009091DB0193FB882780F921E0822780FB86
:1042600093F9EECF0E94931580910D0191E089277B
:1042700080930D0118C027EC01C023EE280F61E0E8
:1042800070E080E090E004C0660F771F881F991FE0
:104290002A95D2F704C061E070E080E090E00E94CF
:1042A00093190E94931581E0089580E0089580E0BD
:1042B0000895CF93C82F8091EB01813079F018F0E9
:1042C0008230D1F184C0A0910E01B0910F018C9188
:1042D000813169F0823209F07CC009C0A0910E01E1
:1042E000B0910F018C91813111F0823249F48C2F01
:1042F0000E94552181111DC08C2F0E949C201AC044
:104300008C2F0E945721811114C0C43179F048F4D8
:10431000CB3079F0C03109F060C082E08093EB01CE
:1043200008C0C93219F0C83321F057C01092EB0110
:1043300054C081E0817053C0C93289F118F5C4318D
:1043400071F1A8F4C73009F046C08AE080931501E6
:1043500094E19093140193E09093130180931201E0
:1043600088E08093110188E28093100134C0CE511F
:10437000C63088F5EC2FF0E0E65DFE4F808180933B
:10438000EA0129C0CE34E9F020F4CB3421F56AE00B
:1043900013C0C13579F0C235F1F461E00DC08091F0
:1043A000EA01882319F01092EA0115C081E0809398
:1043B000EB0115C061E006C08091EA010E94D61FA2
:1043C0000AC06AE08091EA010E944C2004C0109269
:1043D000EB0180E004C081E002C080E0ABCFCF9170
:1043E0000895E1E8F0E080818860808380818160C9
:1043F00080838FB7F89493E09093890090ED909329
:1044000088008FBF0895EFE6F0E0808182608083AE
:104410000895EFE6F0E080818D7F80830895EFE6D8
:10442000F0E0808192E08927808308951F920F92A7
:104430000FB60F9211242F933F934F935F936F9377
:104440007F938F939F93AF93BF93EF93FF9380914D
:10445000EC019091ED0101969093ED018093EC01B8
:10446000811103C082E00E94FC09E091ED01E69514
:10447000E695F0E0E552FA4FE4918091EC018E135D
:1044800003C080E00E94FC09FF91EF91BF91AF91C2
:104490009F918F917F916F915F914F913F912F915C
:1044A0000F900FBE0F901F90189504D06894B11113
:1044B0008DC0089570D088F09F5790F0B92F99273C
:1044C000B751A0F0D1F0660F771F881F991F1AF01F
:1044D000BA95C9F712C0B13081F077D0B1E0089534
:1044E00074C0672F782F8827B85F39F0B93FCCF3B5
:1044F000869577956795B395D9F73EF49095809515
:10450000709561957F4F8F4F9F4F0895E89409C034
:1045100097FB3EF490958095709561957F4F8F4FF6
:104520009F4F9923A9F0F92F96E9BB279395F6950C
:10453000879577956795B795F111F8CFFAF4BB0F8A
:1045400011F460FF1BC06F5F7F4F8F4F9F4F16C0EE
:10455000882311F096E911C0772321F09EE8872F78
:10456000762F05C0662371F096E8862F70E060E034
:104570002AF09A95660F771F881FDAF7880F9695AD
:10458000879597F9089557FD9058440F551F59F096
:104590005F3F71F04795880F97FB991F61F09F3F30
:1045A00079F087950895121613061406551FF2CF59
:1045B0004695F1DF08C0161617061806991FF1CFA9
:1045C00086957105610508940895E894BB276627D0
:1045D0007727CB0197F908950BD078C069D028F0E0
:1045E0006ED018F0952309F05AC05FC01124EECFA9
:1045F000CADFA0F3959FD1F3950F50E0551F629F3E
:10460000F001729FBB27F00DB11D639FAA27F00D2B
:10461000B11DAA1F649F6627B00DA11D661F829F52
:104620002227B00DA11D621F739FB00DA11D621F37
:10463000839FA00D611D221F749F3327A00D611D54
:10464000231F849F600D211D822F762F6A2F112436
:104650009F5750408AF0E1F088234AF0EE0FFF1F89
:10466000BB1F661F771F881F91505040A9F79E3FC0
:10467000510570F014C0AACF5F3FECF3983EDCF315
:10468000869577956795B795F795E7959F5FC1F7FD
:10469000FE2B880F911D9695879597F9089597F9A8
:1046A0009F6780E870E060E008959FEF80EC0895D8
:1046B00000240A9416161706180609060895002401
:1046C0000A9412161306140605060895092E03947B
:1046D000000C11F4882352F0BB0F40F4BF2B11F4EF
:1046E00060FF04C06F5F7F4F8F4F9F4F089597FB10
:1046F000072E16F4009407D077FD09D00E9491236D
:1047000007FC05D03EF4909581959F4F08957095D4
:1047100061957F4F0895EE0FFF1F0590F491E02DF6
:104720000994AA1BBB1B51E107C0AA1FBB1FA617F8
:10473000B70710F0A61BB70B881F991F5A95A9F74A
:1047400080959095BC01CD010895F999FECF92BD59
:1047500081BDF89A992780B50895A8E1B0E042E0BC
:1047600050E00C94CD23262FF999FECF92BD81BD48
:10477000F89A019700B4021639F01FBA20BD0FB69F
:10478000F894FA9AF99A0FBE08950196272F0E947D
:10479000B4230C94B323DC01CB01FC01F999FECFC7
:1047A00006C0F2BDE1BDF89A319600B40D924150B9
:0A47B0005040B8F70895F894FFCFC9
:1047BA000220FE098B0A680A340A010A0101C801AB
:1047CA0028080A03140A404D36399B054E05180578
:1047DA00DF0472048B04A404BD0401020304050669
:0447EA0007080900B3
:00000001FF
